:10000000E9C0A3CB02C101C100C1FFC0FEC0FDC059
:10001000FCC097C6FAC05ACBF8C0F7C057C4F5C0A9
:10002000F4C0F3C0F2C08BC591C5A7C543C642C694
:10003000B8C540C63FC63EC63DC63CC63BC63AC62E
:1000400039C638C606C609C60CC60FC610C611C6C4
:1000500015C624C61AC622C618C617C616C622C694
:1000600029C628C6CAC5CDC5D0C5D3C5D4C5D5C532
:10007000D9C5DFC5B7C5E1C5E4C5E5C5E8C51DC639
:1000800019C618C69FC5A2C5A5C5C3C5C4C5C5C5E3
:10009000C9C5A4C5A7C5ADC5D4C5D5C5D8C50600B5
:1000A000FF0901A101150026FF0075088501950EC5
:1000B0000900B202018502951E0900B20201850302
:1000C000953E0900B202018504957E0900B2020145
:1000D0008506953E0900B20201C01201010100002F
:1000E0000008C016DF05000101020001090222001C
:1000F00001010080640904000001030000000921DF
:1001000001010001223C000705810308000A1201D9
:10011000100102000008C016E10500010102030100
:100120000902430002010080640904000001020288
:100130000100052400100104240202052406000128
:100140000524010301070583030800640904010075
:10015000020A0000000705010208000007058102ED
:100160000800000403090412036F006200640065C4
:100170000076002E00610074003E0348006F0062AC
:10018000006200690065006C0065006B007400721D
:10019000006F006E0069006B0061002E0068007542
:1001A000003A0020004100560052002D0044006F2C
:1001B0000070006500720012036100760072006436
:1001C000006F007000650072000853544B353030EA
:1001D0005F32000011241FBECFE5D4E0DEBFCDBFEB
:1001E00010E0A0E6B0E0E0E3FAE102C005900D9275
:1001F000AE38B107D9F713E0AEE8B0E001C01D9208
:10020000AC3EB107E1F756D011CCFACE2091980060
:10021000FC018381222379F0813019F42AED30E04A
:1002200012C0823021F02EEF30E089E00DC02CEEBC
:1002300030E082E209C0813021F020E231E083E445
:1002400003C02EE031E082E13093010320930003EC
:100250000895FC01808180768032C1F480919800FD
:100260009181882369F0913011F0993009F58281EC
:1002700080939600853011F483E016C081E014C0AD
:1002800090529230A8F41092970010C0803481F4FC
:100290008181813031F482815D9BFECF8CB980E019
:1002A0000895823029F484E0809397008FEF0895B9
:1002B00080E008951F93CF93DF932EE088E190E0D4
:1002C0000FB6F894A89581BD0FBE21BD86E289B90D
:1002D00088E98AB9A49AAC9AA498AC9883B3829519
:1002E0008F70809581708093980081E088BB8FE348
:1002F00087BB88E085BB84E384BB83E182BB81E666
:1003000081BB8B9A20E048EB5BE004C0A895CA0152
:100310000197F1F72150D1F78B9883E083BF81E0FB
:1003200089BF82E88FBD29E02EBD81E090E09BBDB2
:100330008ABD25BD82E083BD08D333D17894A895CA
:1003400082D1E4D4809198008823C9F780916A0013
:1003500084FFF5CFCEE8D0E010E004C089931F5FA2
:10036000183049F0B3D397FFF9CF112321F48091CE
:100370006000882321F310936000612F8EE890E0E5
:100380003FD1DDCF1F93CF93DF93EC01162F8991DF
:10039000F6D21150E1F7DF91CF911F9108950F939D
:1003A0001F93CF93DF93FC01162F90919700992311
:1003B00059F48BE48093F202A1E6B0E087E001906B
:1003C0000D928150E1F724C09330F1F420E06830C1
:1003D00009F021E080919600853031F4818181958A
:1003E000809396003296125080919600882391F166
:1003F00090815D9BFECF9CB98F5F115019F4809363
:1004000096002CC03196F2CF892F8150823010F0A7
:1004100021E024C000E0683009F001E0913011F0E3
:10042000EF0109C0818180939600EF01229612505E
:1004300082E08093970080919600882371F08881F4
:100440009ED280919600815080939600115029F0A1
:100450002196F1CF1092960001C0202F822FDF91BC
:10046000CF911F910F910895FF920F931F93CF93F8
:10047000DF938C01F62E90919700992351F4D801C7
:10048000E1E6F0E087E001900D928150E1F727E08E
:1004900081C09430E9F420E011C0E92FF0E0EE5D76
:1004A000FC4F3281892F8F5F80932203883C10F0AC
:1004B00010922203F80131938F012F5F2F1508F05E
:1004C00069C09091220380912303981731F762C08D
:1004D0009330B1F580919600853019F0D801262F20
:1004E00012C0F80181939091230380912203292F58
:1004F000281B981708F42853DF012D932F2D225025
:1005000081E08093960080919600882309F441C091
:100510009091220380912303981789F1E92FF0E04D
:10052000EE5DFC4F3281892F8F5F80932203883CE0
:1005300010F0109222033C93215059F11196E8CF0C
:10054000892F8150823018F5913019F0E801162F6B
:100550000FC080919600E8018993ACD291118FEF82
:10056000F801818321961F2D125082E0809397001D
:1005700080919600882369F0A9D297FF03C010925A
:10058000960007C08883115021F02196F5CF20E016
:1005900001C02F2D822FDF91CF911F910F91FF90DE
:1005A000089585B7836085BF8BB780648BBF83EC6C
:1005B0008093F2028093E70208951F93DC01162FC7
:1005C00080916B0084FF0AC08091E70298E8892738
:1005D0008093E702912FE8EEF2E007C08AE580936E
:1005E0006B00F8CF8D91819391509923D9F7612FAA
:1005F00088EE92E0A6D81C5F10936B001F910895BF
:100600001F93DC01162F80916A0084FF0AC080913D
:10061000F20298E889278093F202912FE3EFF2E04B
:1006200007C08AE580936A00F8CF8D91819391503D
:100630009923D9F7612F83EF92E083D81C5F109341
:100640006A001F9108950F931F93CF93DF936091DA
:10065000020316160CF0C6C063508091FF02CCE076
:10066000D0E0C81BD109CA5FDC4F8091FE02803107
:1006700018F4CE0187DEB4C08D3209F096C08AE549
:1006800080936900683009F0A3C08881807609F002
:100690007AC01092E5028981882359F41092E6020B
:1006A00085EE92E0909301038093000320E892E0AE
:1006B00075C0853021F48A8180930303FDC08630A4
:1006C00009F042C08B81813071F1823061F1833059
:1006D00041F58A81882349F483E691E090930103F0
:1006E0008093000320EC94E059C0813019F487E630
:1006F00091E010C0823049F489E791E090930103C2
:100700008093000320EC9EE349C0833009F0D6C0FB
:1007100087EB91E0909301038093000320EC92E13A
:100720003DC0813229F4CE0171DD982F20EC2FC01D
:10073000823209F0C3C08EE990E090930103809368
:10074000000320EC9CE32AC0883019F485E093E094
:100750000AC0893021F48A8180930503ADC08A30B4
:1007600049F485EE92E0909301038093000320E822
:1007700091E014C08B3009F09FC083EC8093F202AB
:100780008093E70299C0CE0164DD982F20E89F3F57
:1007900029F4888187FD9E812F771DC08F81882352
:1007A000D1F48E818917C0F016C08091990087FD21
:1007B0000FC0CE01F4DD8F3F21F48EE180936900FC
:1007C00004C0882311F020E004C020E08FEF04C0B3
:1007D00020E880E001C0892F209399008093680071
:1007E000109202038091690084FF5BC080916800D1
:1007F0008F3F09F456C0182F893008F018E0811B8C
:10080000809368008091990080FD02C00BE401C0D4
:1008100003EC8F5F8093990087FF26C0209100032F
:100820003091010386FD05C0D901912FEDEDF2E075
:1008300011C0ADEDB2E080E090E006C0F901E80F34
:10084000F91FE491ED9301961817C1F705C08D913A
:10085000819391509923D9F7F901E10FF11DF0939C
:100860000103E093000309C0112339F0612F8DEDDE
:1008700092E0FADD182F893060F4612F8DED92E05F
:1008800060D7912F9C5F183041F08FEF8093680004
:1008900004C08FEF809368009EE10093DC02909388
:1008A00069009AE080B38C7061F49150D9F710928E
:1008B00003031092FD0205C020E801C020EC90E087
:1008C0006DCFDF91CF911F910F91089578941F9272
:1008D0000F920FB60F9211242F933F938F939F93F4
:1008E00024B135B187B18F70D9F488E393E0821BCE
:1008F000930B25E0880F991F2A95E1F7865D9E4F9F
:10090000181619061CF081E090E006C021E08B3932
:10091000920714F08AE991E09BBD8ABD81EC0AC080
:10092000285F3F4F84E0369527958A95E1F720931D
:10093000800080EC87B9369A9F918F913F912F91DB
:100940000F900FBE0F901F90189580EC87B98DE81F
:1009500086B9369A089580911C0390911D03A09149
:100960001E03B0911F030196A11DB11D80931C03AE
:1009700090931D03A0931E03B0931F030895282F87
:1009800080912103882321F41092B4011092B301C5
:100990008091B3019091B401009761F42B3109F07B
:1009A00085C020939A0081E090E09093B4018093F9
:1009B000B3017CC031E08931930708F073C0FC01BA
:1009C000E656FF4F2083FC013196F093B401E0938B
:1009D000B301E430F105B1F480919D008093B5013D
:1009E00080919C008093B6018091B5019091B601F1
:1009F00006969093B6018093B5018A51914008F410
:100A000055C050C0E530F10521F42E3009F04AC040
:100A10004DC0E530F10508F449C08091B5019091D1
:100A2000B601E817F90709F041C090E0AAE9B0E083
:100A300003C08D91982731973097D9F71092B40160
:100A40001092B301992321F481E08093B7012EC065
:100A500080EB8093BD018093BE018BE18093B80150
:100A600080919B008093B9011092BA0182E080933B
:100A7000BB018EE08093BC011092D2021092D10291
:100A800088E090E09093D4028093D30290E0E8EB6A
:100A9000F1E002C08191982731E0EF3BF307D1F7F5
:100AA000908304C01092B4011092B30188EC80933B
:100AB000210308952091D3023091D4028091D10274
:100AC0009091D202281B390BC90108952091D302BD
:100AD0003091D4022115310519F4EFEFFFEF19C061
:100AE0008091D1029091D202FC01E854FE4FE08146
:100AF00001969093D2028093D1028217930740F01F
:100B00001092D4021092D3021092D2021092D1020B
:100B1000F0E0CF010895CF93DF93C2E0D0E0809161
:100B20009F008093BD011092BE0190E0FC013197BF
:100B3000EC33F10508F0BEC0ED5EFF4F099469EC9F
:100B400071E08FEB91E06BD7CBE0B7C02091A100B3
:100B5000E091A000E63939F485B5922F9770887F2F
:100B6000982B95BD03C0E73909F423BDF0E0EF7180
:100B7000F070E459FF4F2083A0C0E091A000E63957
:100B800019F4E5B5E7700AC0E73911F4E3B506C01A
:100B9000F0E0EF71F070E459FF4FE081E093BF01A6
:100BA00026C08091A00080931F038091A1008093B4
:100BB0001E038091A20080931D038091A300809367
:100BC0001C037BC080EA90E0EAD277C080EA90E024
:100BD0000DD173C080EA90E0DBD26DC080EA90E076
:100BE000A5D169C080EA90E01FD18093BF01C3E026
:100BF00064C080EA90E091D15EC080EA90E000D1CC
:100C00005CC080EA90E000D158C080EA90E0B9D2A0
:100C100052C060E003C040E006C061E080EA90E0BE
:100C2000E2D149C041E06EEB71E080EA90E090D102
:100C30003EC080EA90E05BD13EC080EA90E04ED1B9
:100C40003AC003D1D2CF80EA90E017D1CECF1AD1EB
:100C5000CCCF80EA90E0DCD32EC080EA90E0C1D314
:100C60002CC080EA90E06BD426C060E003C040E076
:100C700006C061E080EA90E07ED41DC041E06EEBEA
:100C800071E080EA90E049D312C080EA90E02AD374
:100C90008093BF011092C001C4E00FC080EA90E0D1
:100CA00038D309C06EEB71E080EA90E0C0D2EC016D
:100CB000219603C080EC8093BE018BE18093B80144
:100CC00080919B008093B901D093BA01C093BB017E
:100CD0008EE08093BC011092D2021092D10226962F
:100CE000D093D402C093D3029E012150304090E0B3
:100CF000E8EBF1E004C081919827215030402115A4
:100D00003105C9F79083DF91CF9108958091B701A4
:100D1000882319F01092B701FEDE0895982F96955A
:100D200096958F5F891B80932003809120038823F1
:100D3000E1F70895F89481E080BF82B7789482B794
:100D4000089578941F920F920FB60F9211248F93EB
:100D5000F89480912003882329F08091200381500A
:100D6000809320037894F89480918C008150809334
:100D70008C00882371F489E480938C0078948091AE
:100D80002103882339F0809121038150809321032E
:100D900001C078948F910F900FBE0F901F901895FF
:100DA000982F9F5F86958695981B909320030895B2
:100DB000382F92B39F7992BBC39AC39880E028E002
:100DC000880F8799816067FD906437FD906292BBC0
:100DD000C39A9F79C398215019F0330F660FF0CF53
:100DE00092BBC39AC398C39AC3980895C298BA9AFB
:100DF000AD9A82B38F7982BBC09AAD98C598089599
:100E000081E08093D502089508951F93182F64E020
:100E10008CE4CEDF60E0812F8866CADF60E0812F3E
:100E20008C66C6DF1F910895FC01E081EE2311F46A
:100E300080E009C0E13011F482E105C0E23011F038
:100E400080EC089582E0E1DF089580E1DEDF08951F
:100E50000F931F93182F062F68E08CE4A9DF612FF2
:100E60008CE0A6DF60E0802F8866A2DF60E0802F44
:100E70008C669EDF1F910F910895FC0160E08081D8
:100E8000E7DF089560E180E0E3DF08958091D60216
:100E900087DF06C080912003882311F480E808953D
:100EA000879BF8CF80E008950F931F93182F042F8E
:100EB0008CE47EDF612F8CE27BDF60E0802F846634
:100EC00077DF60E0802F8C6673DFE0DF182F60E053
:100ED0008CE46EDF812F1F910F910895FC018381B7
:100EE0008093D60240E060E28181DEDF0895FC015C
:100EF00083818093D6028081882311F440E009C069
:100F0000813011F440E105C0823011F042E101C0AE
:100F100042E060E48181C8DF0895FC018281809312
:100F2000D60240E060E28181BFDF0895FC0182814A
:100F30008093D6028081882311F440E005C081307F
:100F400011F042E001C040E160E48181ADDF08952D
:100F5000DF92EF92FF920F931F93CF93DF93FC01E9
:100F6000DB01D42E908181811C928C01442311F4E9
:100F700062E001C063E07D010894E11CF11C8CE497
:100F800017DFE80120C02197A89560911C038CE031
:100F90000FDF60911D038CE10BDF60E088E608DF66
:100FA00060E08CE605DFF70181937F01DD2051F4DD
:100FB00060E088E7FDDE60E08CE7FADEF701819310
:100FC0007F012197C8DC2097F1F6F7011082980184
:100FD0002E5F3F4FC901DF91CF911F910F91FF907D
:100FE000EF90DF9008956F927F928F929F92BF92C1
:100FF000CF92DF92EF92FF920F931F93CF93DF93E5
:10100000FC01C62E83818093D602B280E1808B2DB5
:10101000869581958770DD24DA9402C0D69481503C
:101020008823E1F7CC2011F061E102C0D69460E1A1
:101030008F010C5F1F4F8CE4BBDEFF246B2C7724E9
:1010400081E0882E912C86209720A89560911C0322
:101050008CE0AEDEE80121968114910461F1F80183
:1010600060818E018CE2A4DECC2031F060E08DE660
:101070009FDE60E08CE60AC0FE0161918F018CE387
:1010800097DE60E08DE794DE60E08CE791DE809192
:101090001C038F5F8D21E1F5B7FE3AC060911D03FF
:1010A0008CE186DE60E084E683DE60E08CE680DE54
:1010B000EDDEF82E2DC060911D038CE179DEF80184
:1010C00060818E018CE274DECC2049F060E08DE618
:1010D0006FDE60E084E66CDE60E08CE614C060E009
:1010E00084E666DE60E08CE663DED0DEF82E8823E0
:1010F000D9F4FE0161918F018CE35ADE60E084E750
:1011000057DE60E08CE754DEC1DEF82E882361F400
:1011100022DCCC2011F4EA9419F0EA9409F095CF7E
:10112000892811F066FE03C060E08CE441DE8F2D5B
:10113000DF91CF911F910F91FF90EF90DF90CF90B3
:10114000BF909F908F907F906F9008951F93182F5E
:1011500060E88CE42DDE60E084E62ADE60E08CE668
:1011600027DE8091D602882319F090DE182F03C065
:10117000812FD4DD10E060E08CE41ADE812F1F9116
:101180000895FC0181818093D6028AE0DFDF089513
:10119000FC0180818093D6028181D8DF089510926E
:1011A000D502C59A85B58F7E85BDAD9AC0988F9AB8
:1011B00087E0C0DDAD98BA98C29A82E0BBDD8F9817
:1011C00088E3B8DD0895DF92EF92FF920F931F93AB
:1011D000CF93DF93EC01E62ED090D702F89405B3BD
:1011E0000F7E10E018C0188188E0F82E17FD00610E
:1011F00005BB78948D2D9EDDF894AA9A110F0F7E71
:101200009B9B116078948D2D95DDF894AA98FA94A3
:1012100069F72196EA94EE2031F77894812FDF91D7
:10122000CF911F910F91FF90EF90DF900895AF92B3
:10123000BF92CF92DF92EF92FF920F931F93CF93C3
:10124000DF93EC015B0188811A81811708F4182F64
:10125000612FCE010396B7DF75010894E11CF11CE4
:1012600000E0C12EDD2412C02C0D3D1D2D5F3F4F2F
:1012700061E0CE01820F931FA6DF982F89810817A6
:1012800018F4F70191937F01A8950F5F202F30E0AC
:10129000888190E08C199D09281739072CF30BC021
:1012A0001092D80261E088ED92E08DDFF701819322
:1012B0007F01A8950F5F8981081790F3F5011082CF
:1012C000F7011082298130E02E5F3F4FC901DF9185
:1012D000CF911F910F91FF90EF90DF90CF90BF9033
:1012E000AF9008951F93CF93DF93EC01688101962F
:1012F0006ADF182F8881843038F464E0681B90E03E
:1013000001968C0F9D1F5FDF812FDF91CF911F9181
:10131000089564E058DF80E00895AF92BF92CF92C5
:10132000DF92EF92FF920F931F93CF93DF93EC0125
:101330007B01C42E1092DB02442389F480911F03A9
:1013400087FF0DC08DE48093D8021092D90280915E
:101350001E038093DA0264E088ED92E034DF988126
:10136000898157010894A11CB11CF7011082DA8011
:10137000EC0100E010E01FC0A89580911D03809350
:10138000D90280911C038093DA02CC2041F400FF43
:1013900003C0F8E0DF2A03C087EFD82201C0DBDA00
:1013A000D092D80264E088ED92E00DDFF5018193E0
:1013B0005F010F5F1F4F0C171D07F0F2EC0EFD1EB3
:1013C000F70111829E012E5F3F4FC901DF91CF913E
:1013D0001F910F91FF90EF90DF90CF90BF90AF9053
:1013E00008950F931F938C0185B38B7E85BBAD9AB7
:1013F000F801808193DC85B58F7E85BDC498BC9A49
:10140000AD98C598F801818189DC1F910F910895ED
:10141000DF92EF92FF920F931F93CF93DF93EC0134
:10142000498180918400849902C08DE01CC088238A
:1014300011F0813019F41092D70217C0823011F4E4
:1014400081E011C0833011F482E00DC090E001967C
:101450009C01359527953595279534E09595879589
:101460003A95E1F7820F8093D702C59A85B38B7EB8
:1014700085BBAD9ABC98C49A85B5806185BD842F23
:101480004DDC8091D70256DCAD988091D70252DCBA
:10149000AD9A8A8143DC27E0E22EF12CEC0EFD1E92
:1014A00010E294E0D92E1CC0A8956E81C7018BDE96
:1014B000082F8E81843038F46D2D681B90E00796DC
:1014C0008C0F9D1F80DE8D81081711F480E018C0FD
:1014D000AA9A8091D7022EDCAA988091D7022ADCA2
:1014E000115010F785B38B7E85BBAD9A80E016DC7A
:1014F00085B58F7E85BDC498BC9AAD98C59880ECA3
:10150000DF91CF911F910F91FF90EF90DF900895A1
:101510001F9346DC10EF06C080912003882311F44E
:1015200081E80BC01093D8021092D90264E088EDD4
:1015300092E049DE80FDF0CF80E01F910895FF9298
:101540000F931F938C01FC01F08064E002963BDE58
:10155000F8018181882341F0F9E0FF1510F06AE07D
:10156000F62E8F2DD5DF03C08F2DD8DB80E01F91A5
:101570000F91FF9008956F927F928F929F92AF92FA
:10158000BF92CF92DF92EF92FF920F931F93CF9370
:10159000DF93EC01662EF88019818A8180FD04C0FA
:1015A000E4E07E2E08E003C070E2772E00E46620BF
:1015B00099F480911F0387FF0FC08DE48093D802B8
:1015C0001092D90280911E038093DA021092DB02FE
:1015D00064E088ED92E0F7DDC12EDF2C460108942F
:1015E000810891085E01EE24FF245CC0A8958091DB
:1015F0001D038093D90280911C038093DA02F501C8
:1016000081858093DB021C81662021F4177FE0FE38
:1016100002C01860A0D91093D80264E088ED92E06F
:10162000D2DD8A8180FF0CC0E814F90490F187FFB5
:1016300030C08D818093D80264E088ED92E0C3DDF4
:101640009A81872D8923F1F0F50111858F81181773
:10165000F1F088851817D9F08E81877FE0FC8860CB
:101660008093D8028B819CDB06C080912003882365
:1016700011F480E80FC064E088ED92E0A4DD8117EA
:10168000A1F707C0902319F08B8142DF03C08B8143
:1016900045DB80E00894A11CB11C882341F4089428
:1016A000E11CF11CEC14FD0408F4A0CF80E0DF91F4
:1016B000CF911F910F91FF90EF90DF90CF90BF904F
:1016C000AF909F908F907F906F9008951F920F9290
:1016D0000FB60F9211242F938F939F93EF93FF9345
:1016E0002CB1E09123039E2F9F5F983C08F090E07F
:1016F00080912203981731F0F0E0EE5DFC4F2283D9
:1017000090932303FF91EF919F918F912F910F90D1
:101710000FBE0F901F901895A82FB92F80E090E072
:1017200041E050EA60956F5F58F42D9138EF8227C1
:101730009795879510F0842795273F5FC8F3F3CFDF
:101740000895EADF8D939D930895CF93CFB7CF93FC
:10175000839BFECF839B09C0839B07C0839B05C0EF
:10176000839B03C0839B01C0A6C0DF93C091FF028F
:10177000DD27CA5FDC4F839B02C0DF91EBCF2F9345
:101780000F931F9300B32FEF03FB20F94F933F9369
:1017900010B34FEF012703FB21F93BE031C04E7F2F
:1017A000012F10B3216028C0102F4D7F2260000050
:1017B00000B329C04B7F2460012F000010B32BC061
:1017C00010B3477F28602AC04F7E00B320612CC031
:1017D0004F7D10B320622FC04F7B00B3206432C016
:1017E000422700B349934FEF0000102713FB20F965
:1017F00010B31C70C9F1297F91F2012703FB21F975
:1018000000B3237F89F2315058F1102713FB22F9DE
:1018100010B3277E79F2012703FB23F92F7C81F295
:1018200000B3102713FB24F92F7971F200C010B315
:10183000012703FB25F92F7359F200C000B31027CD
:1018400013FB26F9223040F200C010B3012703FB3E
:1018500027F9243028F64F77206810B30000F9CF1D
:1018600010E41ABF00271CC03B503195C31BD04069
:1018700010E41ABF0881033C11F10B3401F12091EF
:10188000FD021981110F1213EDCF4A81441F093651
:1018900059F10D3211F0013E29F74F7009F0042F74
:1018A000009304033F914F911F910F912F91DF916E
:1018B000CAB7C6FD4DCFCF91CFBFCF91189500913C
:1018C0000403002379F3109102031123F9F5343056
:1018D000FAF1309302030093FE021091FF023BE005
:1018E000311B3093FF0234C000910203013074F5C4
:1018F0000AE54F7049F43091690034FD2BC0009324
:101900006900CCEDD2E02AC0433049F030916A0042
:1019100034FD20C000936A00C2EFD2E01FC03091B6
:101920006B0034FD17C000936B00C7EED2E016C009
:10193000052710E002BB1FC0052722C0052727C0CE
:1019400005272CC0052710E002BB33C04AE503C0C1
:1019500042ED01C0432FC4E1D0E032E011B31C607E
:10196000939A02B311BB5F935CE020E820FF052748
:1019700002BB279517951C3FD8F620FF0527279512
:1019800002BB17951C3FC0F620FF0527279517952A
:1019900002BB1C3F98F620FF0527279517951C3F93
:1019A00002BB70F600C0499120FF052702BB2795B6
:1019B00017951C3F38F620FF0527279502BB179582
:1019C0001C3F38F520FF05272795179502BB1C3FC4
:1019D00010F520FF0527279517951C3F02BBE8F45B
:1019E000242F3A9519F6037F5F9102BB10910303F0
:1019F000110FC651D04011F01093FD0210E41ABF30
:101A0000086011B3137F402F437F02BB11BB42BB61
:101A100049CF0527D3CF0527D8CF0527DDCFFB0139
:101A2000DC0105900D920020E1F70895F894FFCFB6
:101A30000180250000000008FF5A5A5A00000000EB
:101A4000000000000000000000000000010204008F
:0E1A5000320001800200AA0000000000010028
:00000001FF
